:020000020000FC
:020000005EC0E0
:02001800BEC167
:02003C0024C2DC
:020080008FC22D
:0200B4000FC378
:1000BC00BEC201E20EBF0FEF0DBF07E104B908E0AD
:1000CC0005B901E00DBD00E50CBD289A2C980F9ADE
:1000DC0017980000179A0CE000936A0000E20DBB21
:1000EC00259A269A2D982E982227992789E250E056
:1000FC0070E000E0A02EB02EA89500E004BF0EE149
:10010C000093600000E0009360000BEA0093640031
:10011C000FE30093650000E900BF00E20093B60016
:10012C0006E00093B1000091B6000F71E1F707E013
:10013C0007BB01E00093700040E81CD1C6D003EC73
:10014C00289812D1002710D1289A00EE28980CD1AB
:10015C0000E50AD1289A01EE289806D10BEB04D1C0
:10016C00289A02EE289800D103ECFED0289A03EED0
:10017C002898FAD004EAF8D0289A08EC2898F4D0F9
:10018C0005E3F2D0289A05EC2898EED000E8ECD0E4
:10019C00289A0CEE2898E8D008E3E6D0289A0EEEC0
:1001AC002898E2D002E0E0D0289A0DEE2898DCD016
:1001BC0000E8DAD0289A0FE82898D6D0289A0EECC6
:1001CC002898D2D008E0D0D0289AA8950EE10093B8
:1001DC00600008E2009360000FEF0CBB78942C9A3F
:1001EC0007E003BF65E088950000000000006A95F9
:1001FC00D1F7002703BF2C9848E2BCD06CD0A5D017
:10020C0030EA4FEFB7D0863D41F13A95D1F76CD03B
:10021C00E6CF6AD065D100E00093A1000093720094
:10022C000000000000007230D9F300E00093910050
:10023C0000932101009381000093710000937300DF
:10024C00009380000BEA009364000FE300936500B9
:10025C002D982E9850E070E0C2CF03EA0093640012
:10026C0007E00093650003EA0093800000E0009330
:10027C0089000093880000938B0000938A000AE0A9
:10028C00009381000ED10000000000005130D9F322
:10029C0000E00093A5000093A40001E0009372001D
:1002AC0002E00093A1000000000000008932D9F7A1
:1002BC0088270000000000008932D9F78827000049
:1002CC00000000008932D9F7A4CF02EC28984CD05A
:1002DC0008E04AD0289A01E8289846D000E044D09B
:1002EC00289A0830C1F7089502EC28983DD003E015
:1002FC003BD0289A000000000000000001E828987C
:10030C0033D000E031D0289A083071F7089502EC10
:10031C0028982AD009E028D0289A01E8289824D0D7
:10032C0000E022D0289A0930C1F7089502EC2898F1
:10033C001BD009E119D0289A01E8289815D000E0C3
:10034C0013D0289A0931C1F7089502EC28980CD0E3
:10035C0006E10AD0289A01E8289806D000E004D0DB
:10036C00289A0631C1F708950EBD0DB507FFFDCFD4
:10037C000EB5089500000000000000000000000011
:10038C00000000004A95B1F708950F930FB70F9333
:10039C000FE82898E9DF289A01E82898E5DF00E0C3
:1003AC00E3DF289A063139F0013129F00F31A1F33E
:1003BC00023191F336C0002400E22898D5DF00E02A
:1003CC00D3DF003171F500E0CFDF00E0CDDF00E0DE
:1003DC00CBDF003059F1023021F500E0C5DF00E041
:1003EC00C3DF00E0C1DF00E0BFDF00E0BDDF0835A8
:1003FC00C1F400E0B9DF0B3BA1F400E0B5DF002E47
:10040C0000E0B2DF073669F400E0AEDF013C49F4EE
:10041C0000E0AADF0A3829F400E0A6DF0F3909F45E
:10042C009029289A0F910FBF0F91189500E09CDF2F
:10043C0000E09ADF00E098DF00E096DF00E094DF58
:10044C00043579F700E090DF0B3B59F700E08CDFC7
:10045C00002E00E089DF0B3A21F700E085DF06343F
:10046C0001F700E081DF0733E1F600E07DDF023DBC
:10047C00C1F6802DAA24BB24D4CF000000000000BC
:10048C000F930FB70F9301E0A00E0027B01E28F0BA
:10049C00A8950F910FBF0F91189500000000000058
:1004AC00FCCF00E000939500009394000EE40093C1
:1004BC00990000E20093980002E00093710005E0BF
:1004CC00009391000FEF009389000FEF00938800C9
:1004DC0000E000938B0000938A0051E070E00895D7
:1004EC0000E000932501009324010EE40093290100
:1004FC0000E20093280102E00093730005E00093F2
:10050C0021010FEF00938B0000938A0000E0009311
:10051C0089000093880072E050E008955330D1F0C8
:10052C005430C1F000E0009395000093940002E079
:10053C000093990003EA0093980002E00093710085
:10054C000AE00093910000E000938900009388007A
:10055C00B0E2AA2753E008957530D1F07630C1F09F
:10056C0000E0009325010093240105E0009329018C
:10057C0003EA0093280102E0009373000AE0009361
:10058C00210100E000938B0000938A00D0E2CC277D
:10059C0075E008950F930FB70F93513091F05330CE
:1005AC00F1F05430E1F000E0009391000093710001
:1005BC00009389000093880050E00F910FBF0F91BA
:1005CC00189500E00093910000937100009389004E
:1005DC000093880050E00F910FBF0F911895FD010B
:1005EC0005901590DF01F83241F0109289000092CD
:1005FC0088000F910FBF0F911895543051F0B0E255
:10060C00AA2710928900009288000F910FBF0F91BA
:10061C00189500E0009391000093710000938900FD
:10062C000093880050E00F910FBF0F9118950F9316
:10063C000FB70F93723091F07530F1F07630E1F026
:10064C0000E0009321010093730000938B00009352
:10065C008A0070E00F910FBF0F91189500E0009386
:10066C0021010093730000938B0000938A0070E0CB
:10067C000F910FBF0F911895FE0105901590EF018A
:10068C00F83241F010928B0000928A000F910FBF4C
:10069C000F911895763051F0D0E2CC2710928B0048
:1006AC0000928A000F910FBF0F91189500E00093F4
:1006BC0021010093730000938B0000938A0070E07B
:1006CC000F910FBF0F9118950F930FB70F93903099
:1006DC0059F09130A1F09230B1F09330D1F09927CC
:1006EC000F910FBF0F911895533019F0753029F0F9
:1006FC00F6CF54E0753009F0F2CF76E0F0CF0EDF94
:10070C007530D9F3ECCF28DF533009F0E8CF54E043
:08071C00E6CF04DF21DFE3CF8B
:1020000000000000000000000000000000000000D0
:1020100001000100010001000100020002000200B5
:102020000200030003000300040004000500050093
:102030000600060006000700080008000900090065
:102040000A000A000B000C000C000D000E000F002F
:102050000F001000110012001300130014001500EF
:1020600016001700180019001A001B001C001D00A4
:102070001E001F0020002100220023002500260052
:102080002700280029002B002C002D002E003000F6
:1020900031003200340035003700380039003B0091
:1020A0003C003E003F004100420044004600470023
:1020B00049004A004C004E004F00510053005400AC
:1020C000560058005A005B005D005F00610063002D
:1020D0006500660068006A006C006E0070007200A7
:1020E0007400760078007A007C007E008000820018
:1020F0008400860089008B008D008F009100930082
:10210000960098009A009C009F00A100A300A600E2
:10211000A800AA00AD00AF00B100B400B600B8003E
:10212000BB00BD00C000C200C500C700CA00CC0093
:10213000CF00D100D400D600D900DB00DE00E100E2
:10214000E300E600E800EB00EE00F000F300F6002C
:10215000F800FB00FE0000010301060109010B016C
:102160000E0111011401160119011C011F012201A8
:10217000250127012A012D013001330136013901E2
:102180003B013E014101440147014A014D0150011B
:102190005301560159015C015F016201650168014B
:1021A0006B016E017101740177017A017D0180017B
:1021B0008301860189018C018F01920195019801AB
:1021C0009B019E01A101A501A801AB01AE01B101D6
:1021D000B401B701BA01BD01C001C401C701CA0100
:1021E000CD01D001D301D601D901DD01E001E30128
:1021F000E601E901EC01EF01F201F601F901FC0150
:10220000FF010202050208020C020F02120215026F
:1022100018021B021E022102250228022B022E0296
:102220003102340237023A023E02410244024702BE
:102230004A024D0250025302560259025D026002E8
:102240006302660269026C026F0272027502780212
:102250007B027E028102840287028A028D02900242
:102260009302960299029C029F02A202A502A80272
:10227000AB02AE02B102B402B702BA02BD02C002A2
:10228000C302C502C802CB02CE02D102D402D702D9
:10229000D902DC02DF02E202E502E802EA02ED0214
:1022A000F002F302F502F802FB02FE020003030350
:1022B000060308030B030E0310031303160318038E
:1022C0001B031D0320032303250328032A032D03D7
:1022D0002F0332033403370339033C033E03410326
:1022E0004303460348034A034D034F03510354037A
:1022F000560358035B035D035F03620364036603D5
:1023000068036B036D036F03710373037503780335
:102310007A037C037E03800382038403860388039D
:102320008A038C038E03900392039403960398030D
:1023300099039B039D039F03A103A303A403A60387
:10234000A803AA03AB03AD03AF03B003B203B40306
:10235000B503B703B803BA03BC03BD03BF03C0038F
:10236000C203C303C503C603C703C903CA03CC031F
:10237000CD03CE03D003D103D203D303D503D603B9
:10238000D703D803D903DB03DC03DD03DE03DF035C
:10239000E003E103E203E303E403E503E603E70309
:1023A000E803E903EA03EB03EB03EC03ED03EE03BD
:1023B000EF03EF03F003F103F203F203F303F4037B
:1023C000F403F503F503F603F603F703F803F80344
:1023D000F803F903F903FA03FA03FB03FB03FB0316
:1023E000FC03FC03FC03FC03FD03FD03FD03FD03F1
:1023F000FD03FE03FE03FE03FE03FE03FE03FE03D6
:10240000FE03FE03FE03FE03FE03FE03FE03FE03C4
:10241000FD03FD03FD03FD03FD03FC03FC03FC03BF
:10242000FC03FB03FB03FB03FA03FA03F903F903C1
:10243000F803F803F803F703F603F603F503F503CF
:10244000F403F403F303F203F203F103F003EF03E5
:10245000EF03EE03ED03EC03EB03EB03EA03E90305
:10246000E803E703E603E503E403E303E203E10330
:10247000E003DF03DE03DD03DC03DB03D903D80362
:10248000D703D603D503D303D203D103D003CE039E
:10249000CD03CC03CA03C903C703C603C503C303E3
:1024A000C203C003BF03BD03BC03BA03B803B70331
:1024B000B503B403B203B003AF03AD03AB03AA0388
:1024C000A803A603A403A303A1039F039D039B03E7
:1024D0009903980396039403920390038E038C034D
:1024E0008A03880386038403820380037E037C03BC
:1024F0007A0378037503730371036F036D036B0332
:1025000068036603640362035F035D035B035803B0
:102510005603540351034F034D034A034803460334
:10252000430341033E033C033903370334033203BF
:102530002F032D032A0328032503230320031D0350
:102540001B0318031603130310030E030B030803E6
:10255000060303030003FE02FB02F802F502F30286
:10256000F002ED02EA02E802E502E202DF02DC022A
:10257000D902D702D402D102CE02CB02C802C502D0
:10258000C302C002BD02BA02B702B402B102AE0277
:10259000AB02A802A502A2029F029C029902960227
:1025A000930290028D028A028702840281027E02D7
:1025B0007B027802750272026F026C026902660287
:1025C000630260025D0259025602530250024D023C
:1025D0004A024702440241023E023A0237023402F2
:1025E00031022E022B022802250221021E021B02AA
:1025F0001802150212020F020C0208020502020262
:10260000FF01FC01F901F601F201EF01EC01E90122
:10261000E601E301E001DD01D901D601D301D001DA
:10262000CD01CA01C701C401C001BD01BA01B70192
:10263000B401B101AE01AB01A801A501A1019E0148
:102640009B019801950192018F018C0189018601FE
:10265000830180017D017A017701740171016E01AE
:102660006B016801650162015F015C01590156015E
:10267000530150014D014A014701440141013E010E
:102680003B0139013601330130012D012A012701B7
:10269000250122011F011C0119011601140111015C
:1026A0000E010B010901060103010001FE00FB0000
:1026B000F800F600F300F000EE00EB00E800E600A2
:1026C000E300E000DE00DB00D900D600D400D1003A
:1026D000CF00CC00CA00C700C500C200C000BD00CA
:1026E000BB00B800B600B400B100AF00AD00AA0056
:1026F000A800A600A300A1009F009C009A009800DB
:102700009600930091008F008D008B008900860059
:102710008400820080007E007C007A0078007600D1
:102720007400720070006E006C006A006800660041
:102730006500630061005F005D005B005A005800A7
:1027400056005400530051004F004E004C004A0008
:102750004900470046004400420041003F003E005F
:102760003C003B00390038003700350034003200AF
:10277000310030002E002D002C002B0029002800F5
:1027800027002600250023002200210020001F0032
:102790001E001D001C001B001A0019001800170065
:1027A0001600150014001300130012001100100091
:1027B0000F000F000E000D000C000C000B000A00B3
:1027C0000A000900090008000800070006000600CA
:1027D00006000500050004000400030003000300D8
:1027E00002000200020002000100010001000100DD
:1027F00001000000000000000000000000000000D8
:00000001FF
